:020000040000FA
:100000002500520A34000802090143064E0A480935
:100010006C006D00540220094F090B02EC01000234
:100020001401030794012000AD024306A802430611
:10003000E9030C0A14021C0A1701370006004E0AD5
:100040005701370006004E0A6C002B00FF0CEB0135
:100050000307EC0103074E0A030C2900DF0C3209E9
:10006000260A69002800E70CE8016902FC0C030776
:100070003D0AE8010306390AE8010400E903390AE8
:100080000806420A2807460A0000460A000803003C
:1000900068026902A8024306A9020008C404A40475
:1000A00004000008640083065C0A63065C0A13020D
:1000B0000200170206000008FF0C33003700180C7E
:1000C00036006704D00C02002500080C370006003B
:1000D00066007E0004000A0C9E0003067F0A0605E7
:1000E0000602170417020600640C2409060406021F
:1000F000170417020600640C2409FE036A0A7D0037
:100100001D022B00010C28006900060C2400010CC4
:1001100002091D022B00010C28006900060C2400B6
:10012000020C02091D022B00010C28006900060CBC
:100130002400040C0209040CFD010307800A7E0060
:10014000FF0C2A001E028A003D001D022B00010C3C
:1001500028006900060C2400010C02091D022B0076
:10016000010C28006900060C2400020C02091D0283
:100170002B00010C28006900060C2400040C020965
:10018000040CFE010307A00A060506021704170265
:100190000600260506023704170206004605060279
:1001A000570417020600010C2C002C0C250906042C
:1001B0000602170417020600260406023704170277
:1001C000060046040602570417020600010C2C0024
:1001D0002C0C250906050602170417020600260541
:1001E00006023704170206004605060257041702E6
:1001F0000600010C2C002C0C25090604060217042D
:1002000017020600260406023704170206004604F9
:100210000602570417020600010C2C002C0C2509BD
:100220007D001D022B00010C28006900060C240033
:10023000010C0209080CFD010307110B7F000400EB
:10024000030C9F000306960B7D00FF0C2A001D0285
:100250008A003E001E022B00010C28006900060CDB
:100260002400010C02091D022B00010C280069006A
:10027000060C2400020C0209080CFD010307250BE3
:100280007D00FF0C2A001D028A003E001E022B008A
:10029000010C28006900060C2400020C02091D0252
:1002A0002B00010C28006900060C2400040C020934
:1002B000080CFD010307410B7D00FF0C2A001D0205
:1002C0008A003E001E022B00010C28006900060C6B
:1002D0002400040C02091D022B00010C28006900F7
:1002E000060C2400020C0209080CFD0103075D0B3B
:1002F0007D00FF0C2A001D028A003E001E022B001A
:10030000010C28006900060C2400020C02091D02E1
:100310002B00010C28006900060C2400010C0209C6
:10032000080CFD010307790BFF031F0B7E0004007F
:10033000030C9E000306DD0B0605060217041702D8
:100340000600640C2409260506023704170206007D
:10035000640C240906040602170417020600640C44
:10036000240946050602570417020600640C2409F6
:1003700026040602370417020600640C2409260529
:100380000602370417020600640C2409460406021C
:10039000570417020600640C240906050602170418
:1003A00017020600640C240926040602370417020B
:1003B0000600640C2409FE03970B690A4709DE0B4B
:021FFE00FF0FD3
:00000001FF
